S01900006F70656E626C745F73746D3332673037312E7372656300
S31508000000009000209D050008890500088B0500085A
S3150800001000000000000000000000000000000000D2
S315080000200000000000000000000000008D05000828
S3150800003000000000000000008F0500089105000878
S31508000040ED050008ED050008ED050008ED050008BA
S31508000050ED050008ED050008ED050008ED050008AA
S31508000060ED050008ED050008ED050008ED0500089A
S31508000070ED050008ED050008ED050008ED0500088A
S31508000080ED050008ED050008ED050008ED0500087A
S31508000090ED050008ED050008ED050008ED0500086A
S315080000A0ED050008ED050008ED050008ED0500085A
S311080000B0ED050008ED050008ED05000848
S315080000BC10B5064C2378002B07D1054B002B02D024
S315080000CC044800E000BF0123237010BD1000002077
S315080000DC000000002C1D0008044B10B5002B03D0A3
S315080000EC0349044800E000BF10BDC04600000000EC
S315080000FC140000202C1D0008002243088B4274D3E0
S3150800010C03098B425FD3030A8B4244D3030B8B42FE
S3150800011C28D3030C8B420DD3FF22090212BA030C07
S3150800012C8B4202D31212090265D0030B8B4219D3E8
S3150800013C00E0090AC30B8B4201D3CB03C01A524108
S3150800014C830B8B4201D38B03C01A5241430B8B4250
S3150800015C01D34B03C01A5241030B8B4201D30B0339
S3150800016CC01A5241C30A8B4201D3CB02C01A524160
S3150800017C830A8B4201D38B02C01A5241430A8B4223
S3150800018C01D34B02C01A5241030A8B4201D30B020C
S3150800019CC01A5241CDD2C3098B4201D3CB01C01A26
S315080001AC524183098B4201D38B01C01A5241430930
S315080001BC8B4201D34B01C01A524103098B4201D31E
S315080001CC0B01C01A5241C3088B4201D3CB00C01A8B
S315080001DC524183088B4201D38B00C01A5241430803
S315080001EC8B4201D34B00C01A5241411A00D2014628
S315080001FC524110467047FFE701B5002000F006F89B
S3150800020C02BDC0460029F7D076E770477047C0464E
S3150800021C10B501F0EDFA10BD10B501F0F7FA10BDE6
S3150800022C10B5054B1B699B0401D4002010BD00F0CA
S3150800023C3DF80120FAE7C0460008005010B56420C6
S3150800024C00F006F810BD10B500F008F810BD000057
S3150800025C014B18807047C0462C00002010B501F0E1
S3150800026C79FA0F4B1B68984211D30E4B1B78002B4F
S3150800027C0ED10C4B01221A70A023DB051F329A6192
S3150800028C01F068FA084B1B881B18054A136010BD49
S3150800029C044B00221A70A023DB0520329A62EFE782
S315080002AC300000202E0000202C000020A023DB05A7
S315080002BC20229A627047000070B588B0142200217B
S315080002CC03A801F025FD164B596B042211435963FB
S315080002DC596B0A400192019A5A6B01252A435A63B3
S315080002EC5B6B2B400293029BA026F605002220216D
S315080002FC300000F0E7FB80239B0103930024049451
S3150800030C059403A9074800F021FB202303930495C1
S3150800031C0594069403A9300000F018FB08B070BDCC
S3150800032C0010024000080050F0B591B020220021C0
S3150800033C08A801F0EDFC344BD96B802080020143F0
S3150800034CD963DA6B02400192019A5A6B01252A434A
S3150800035C5A635B6B2B400093009B04230293022782
S3150800036C039700240494059406940795A026F6058D
S3150800037C02A9300000F054FC082302930397049456
S3150800038C05940694079502A9300000F049FC0894D8
S3150800039CE1235B0209930A940B940C940C230D939A
S315080003AC0E940F94194C08A9200000F06DFDEFF37C
S315080003BC108285F31088A368DB00DB08A36082F340
S315080003CC1088EFF3108285F31088A36810490B4048
S315080003DCA36082F3108823680E4A1340236063686F
S315080003EC0D4A13406360A3682A229343A3602368CB
S315080003FC1D432560054BDB699B02FBD5034BDB696B
S3150800040C5B02F7D511B0F0BD001002400044004065
S3150800041CFFFFFFF1FFFFFFDFFFB7FFFF10B5264A0F
S3150800042C136807218B4305390B431360224B1A6853
S3150800043C07231340022BF9D1204A1168FE330B43CC
S3150800044C13601E4B1B685B05FBD51C4BDA681C49F5
S3150800045C11401C4A0A43DA601968802252040A437E
S3150800046C1A60D968802252050A43DA60134B1B6856
S3150800047C9B01FBD5114A936813490B40936093680B
S3150800048C07218B4305390B4393600C4B9A68382329
S3150800049C1340102BF9D1094CA3680C4A1340A360DE
S315080004AC0B4800F087FD002000F0B0F8636D0C22B5
S315080004BC9343636510BDC0460020024000100240FD
S315080004CC8C80FF1F32400060FFF0FFFFFF8FFFFF9D
S315080004DC0090D00310B500F0C5F8FFF79FFFFFF7A3
S315080004ECEBFEFFF721FFFFF793FEFFF795FEFCE700
S315080004FC00B583B00B4B196C012211431964196CA6
S3150800050C0A400092009ADA6B802149050A43DA639D
S3150800051CDB6B0B400193019BC020C00000F0C2F8B6
S3150800052C03B000BD0010024010B500F0D1FAA024AB
S3150800053CE4052023A3620D4800F024FB200000F0FC
S3150800054C21FB0B4BDA6B0B490A40DA635A6B042115
S3150800055C8A435A635A6B03398A435A63DA6B0648D9
S3150800056C0240DA631A6C8A431A6410BD00080050FC
S3150800057C00100240FFFFFDFFFFFFFFEF7047FEE78D
S3150800058C7047704710B500F081F810BD7047000031
S3150800059C0D488546002103E00C4B5B58435004314B
S315080005AC0B480C4B42189A42F6D30B4A02E000232E
S315080005BC13600432094B9A42F9D3FFF7E7FF01F0AF
S315080005CC83FBFFF787FFFEE7009000203420000826
S315080005DC000000201000002010000020400500201C
S315080005ECFEE7000010B5084B01214942D9620022EA
S315080005FCDA6219631A6399629A6259625A62FFF748
S3150800060C93FF002010BDC0460010024010B5040030
S3150800061C114B1978002901D1012010BDFA20800050
S3150800062CFFF76AFD01000D4B1868FFF765FD00F032
S3150800063C75F800280DD1032C01D90120EDE70130FE
S3150800064C00222100404200F039F8054B1C600020BE
S3150800065CE3E70120E1E7C046040000200000002083
S3150800066C0800002010B5084A116880235B000B436C
S3150800067C13600020FFF7CAFF041E02D001242000D5
S3150800068C10BDFFF735FFFAE700200240034B1B7835
S3150800069C034A11685B1813607047C04604000020B3
S315080006AC3C050020034A136803490B4003431360B7
S315080006BC7047C04600000140FFF9FFFF70B50028DF
S315080006CC11DB8308134EC0339B009D59032420402D
S315080006DCC000FF2214008440A54389010A408240C9
S315080006EC2A439A5170BD0F230340083B9B080633D7
S315080006FC9B00094A944663445C6803221040C00078
S3150800070CFC3215008540AC4389010A4082402243DD
S3150800071C5A60E7E700E100E000ED00E001388023CD
S3150800072C5B0498420FD2094A50600948036A1B02B7
S3150800073C1B0AC02109060B43036200239360073387
S3150800074C1360002070470120FCE7C04610E000E06B
S3150800075C00ED00E030B5054C61690125294361615E
S3150800076C0260BFF36F8F436030BDC0460020024065
S3150800077C084B5B69002B01DB00207047054B064ACA
S3150800078C9A60064A9A605B69002B01DB0020F4E745
S3150800079C0120F2E70020024023016745AB89EFCD23
S315080007AC064B5969802212060A435A615B69002B6B
S315080007BC01DB012070470020FCE7C0460020024000
S315080007CC70B5050000F0CEFF4419134B1B69DB030B
S315080007DC05D500F0C7FFA042F7D3032070BD0E491C
S315080007EC0A690E4B14001C400D4808611A4203D0C6
S315080007FC0C4B5C600120F1E700F0B4FF4519064B81
S3150800080C1B695B0305D500F0ADFFA842F7D303209F
S3150800081CE4E70020E2E7C04600200240FAC30000E5
S3150800082CFBC3000034000020F8B507000C001500C7
S3150800083C1E00144B1B78012B22D0124B01221A7066
S3150800084C00225A60FA208000FFF7BAFF00280DD163
S3150800085C012F0FD02900200001F06EFAFA20800033
S3150800086CFFF7AEFF084A5369BB435361054B002299
S3150800087C1A70F8BD2A0033002000FFF76BFFEDE76E
S3150800088C0220F6E73400002000200240034A536990
S3150800089C03438020400218435061704700200240F1
S315080008AC044A536904480340C9001943034B1943C6
S315080008BC516170470020024007FEFFFF020001004D
S315080008CC70B504000E001F4B1B78012B37D01D4B3F
S315080008DC01221A7000225A60FA208000FFF770FF76
S315080008EC002828D1042363602368042B15D0012320
S315080008FC5B423360A568A368E26894466344AB42DE
S3150800090C14D929006068FFF7CBFFFA208000FFF79F
S3150800091C57FF002809D10135EDE70430FFF7B6FF7C
S3150800092CFA208000FFF74CFF05E03560064A53694C
S3150800093C02218B435361034B00221A7070BD0220AF
S3150800094CFCE7C0463400002000200240F0B5002326
S3150800095C5AE084685F000326BE40B4432600CC6880
S3150800096CBC4034438460446894434A68160901229F
S3150800097C32409A402243426056E0DC080834A40010
S3150800098C265805321A4092000F279740BE430F6926
S3150800099C97403A00324322505AE0032600E00026DC
S315080009ACA64034003C43434E1832920094518022A0
S315080009BCB458EA432600AE434F68FF0301D52C43CF
S315080009CC26003C4C8027E6518426A459260016405E
S315080009DC4F68BF0301D52C432600364C8427E651B5
S315080009EC2468260016404F68FF0201D52C432600C2
S315080009FC304C2660646822404E68B60201D52A003F
S31508000A0C22432C4C626001330C682200DA404FD02A
S31508000A1C01229A40250015401442F4D003244E684E
S31508000A2C3440013C012C94D903224C682240032AF9
S31508000A3C09D0C2685E000324B440A24314008A6835
S31508000A4CB2402243C26003224C682240022A94D048
S31508000A5C04685E0003221700B740BC434F683A404F
S31508000A6CB24022430260C02292024C681442CAD099
S31508000A7C9A0814001834A4000E4EA75903241C40D7
S31508000A8CE4000F26A640B743A026F605B04286D04A
S31508000A9C094EB04208D0094EB04207D0084EB042B3
S31508000AAC00D17AE705267BE7012679E7022677E760
S31508000ABCF0BDC04600180240000400500008005063
S31508000ACC000C0050002A01D0816170478162FCE756
S31508000ADC70B500F047FE0400254A116880235B00B8
S31508000AEC0B431360224B1B685B0506D400F03AFED9
S31508000AFC001B0228F6D9032070BD1D4D8023DB018F
S31508000B0C6B6000F02FFE04000023AB60184B9B684B
S31508000B1C38221A4207D000F025FE001B154B9842C6
S31508000B2CF4D90320E8E7124BC8321A601A6000F0B1
S31508000B3C19FE04000E4B1B689B0106D500F012FE2D
S31508000B4C001B0228F6D90320D6E7094B802252014E
S31508000B5CDA6000229A61013A1A62074B074A1A6050
S31508000B6C074B1868FFF752FD0028C5D00120C3E7CC
S31508000B7C0010024088130000000000200024F40036
S31508000B8C08000020A023DB0598420DD01F4B984285
S31508000B9C14D01F4B98421BD01E4B984222D01E4B8A
S31508000BAC984229D0012008E01C4B5A6A01210A43B5
S31508000BBC5A625A6A8A435A6200207047174B5A6A15
S31508000BCC02210A435A625A6A8A435A620020F4E797
S31508000BDC124B5A6A04210A435A625A6A8A435A625F
S31508000BEC0020EAE70D4B5A6A08210A435A625A6AE8
S31508000BFC8A435A620020E0E7084B5A6A20210A43C6
S31508000C0C5A625A6A8A435A620020D6E70004005090
S31508000C1C00080050000C0050001400500010024050
S31508000C2CF0B5002226E083682C006C436600361962
S31508000C3CB3438E687443234383604368AB43CC68E1
S31508000C4C6C4323434360C6682B006B435F00FF1855
S31508000C5CFC43A446BE430F695F433E43C6604C68DB
S31508000C6C022C16D0046865462C404D686B4323430A
S31508000C7C036001320C682300D34026D0012393402D
S31508000C8C25001D401C42F4D04B68013B012BDAD8D9
S31508000C9CC9E7FF2D0BD8066A1C006C4365432C016B
S31508000CAC641BA6434C69654335430562DAE7466A15
S31508000CBC2D0A2C006C436C4365432C01641BA6431C
S31508000CCC4C69654335434562CCE70020F0BD00000E
S31508000CDC054B9A68120A0F2313409B00034A9A582D
S31508000CEC1F231340D8407047001002407C1D000893
S31508000CFC054B9A68120B072313409B00034A9A5814
S31508000D0C1F231340D840704700100240BC1D000832
S31508000D1C10B50E4BDA6803231340032B13D00C4A79
S31508000D2C0A4CE3681B0A7F2018405043E3681B09EA
S31508000D3C072119400131FFF7DFF9E168490F013145
S31508000D4CFFF7DAF910BD034AEAE7C046001002407D
S31508000D5C0024F40000127A0010B50A4B9A6838235E
S31508000D6C1340082B0CD0102B02D1FFF7D1FF08E04B
S31508000D7C044B1A68D20A072313400348D84000E0EC
S31508000D8C024810BD001002400024F40000127A003C
S31508000D9C10B50400FFF7E0FF2060FFF799FF6060CD
S31508000DACFFF7A6FFA06010BD10B5032803D00C28CA
S31508000DBC2DD0002010BD2C4B5B6D0340000418434E
S31508000DCC2A4B98420FD02A4B984216D0294B984258
S31508000DDC06D0FFF7C1FFFFF77BFFFFF789FFE9E7AF
S31508000DECFFF7BAFFE6E7204B1A688023DB001000F2
S31508000DFC18401A42DED02048DCE71B4BDB6D02227A
S31508000E0C100018401A42D5D080200002D2E7164BA3
S31508000E1C5B6D034000041843184B98420FD0184BCF
S31508000E2C984216D0174B984206D0FFF795FFFFF756
S31508000E3C4FFFFFF75DFFBDE7FFF78EFFBAE70A4BDB
S31508000E4C1A688023DB00100018401A42B2D00A48F0
S31508000E5CB0E7054BDB6D0222100018401A42A9D0E8
S31508000E6C80200002A6E7C0460010024002000300DC
S31508000E7C03000300010003000024F40008000C0022
S31508000E8C0C000C0004000C0070B584B004000D00B6
S31508000E9C0368DB0700D578E003683D4A1A408B687F
S31508000EAC09690B4369690B43E9690B4313430360EF
S31508000EBC4368384A1340EA68134343608368364AE2
S31508000ECC1340AA6913438360344B984213D0344BAE
S31508000EDC98421AD0334B98421BD0334B98421DD0AC
S31508000EEC01202B68E26A0F218A431B041B0C13434F
S31508000EFCE36204B070BD0320FFF756FF002842D00A
S31508000F0C6E68002E0FD10120EBE70C20FFF74CFF83
S31508000F1CF4E701A8FFF73CFF0398EFE701A8FFF7F2
S31508000F2C37FF0398EAE72B68EA690B2B14D8002ECF
S31508000F3C12D0802109028A4210D0FF2213409B004E
S31508000F4C1A4A9958FFF7D8F87308C0183100FFF7F2
S31508000F5CD3F80004000CE0600020C2E7FF2213401F
S31508000F6C9B00124A9958FFF7C7F840007308C01837
S31508000F7C3100FFF7C1F80E4B03404008072210401A
S31508000F8C1843E060E8E70120ABE70120B1E7C0466B
S31508000F9CF369FFEFFFCFFFFFFFFCFFFF00380140AF
S31508000FAC0044004000480040004C0040DC1D00088E
S31508000FBCF0FF0000014B18607047C0460000002087
S31508000FCC72B6704762B6704710B5FFF7F9FF10BDD9
S31508000FDC10B500F0CFFA002800D110BDFFF720F9A4
S31508000FEC0028FAD000F040FCFFF7FCFA00F088FB6A
S31508000FFC00F0C4FA054B1840054B986000F0BEFA91
S3150800100C4468FFF7DFFFA047E7E7C04680FFFF1FEE
S3150800101C00ED00E070B5541EA4B2002A09D04D1C90
S3150800102C461C0B78037000F05EFC30002900220089
S3150800103CF1E770BD70B50500002401E00134E4B297
S3150800104C0D2C17D800F04FFC63001B199B000A499E
S3150800105C5B58AB42F2D86100091989000648411859
S3150800106C49685B18AB42E9D963001A1992008218D1
S3150800107C107A00E0FF2070BD581E000870B50500F8
S3150800108C00240D2C11D800F02EFC63001B199B00B4
S3150800109C074AD3181B7AAB4202D00134E4B2F0E704
S315080010AC630019198900885801E00120404270BD77
S315080010BC581E000870B5050000240D2C12D800F037
S315080010CC12FC63001B199B00074AD3181B7AAB4208
S315080010DC02D00134E4B2F0E76300191989005118FB
S315080010EC486800E0002070BD581E000810B5CB05F6
S315080010FC0BD103688B4201D1012007E002C0802284
S3150800110C9200FFF787FF012000E0002010BDF8B51C
S3150800111CCE46474680B581460068FFF78BFFFF2809
S3150800112C06D1002398464046C0BCB946B046F8BD21
S3150800113CFFF71EFB002500E001353F2D18D8EB0004
S3150800114C4A461268D4184B445E689F6800F0CBFB7D
S3150800115C32003B0021000120FFF766FB8046002881
S3150800116C09D122686368B24207D1BB42E4D004E0D5
S3150800117C0123984601E000239846FFF711FBD2E7B6
S3150800118C70B504000D000F4B984214D00E4B9942C3
S3150800119C0BD10C4E3400002E05D029002000FFF789
S315080011ACA5FF00280CD0300070BDFFF7B0FF012852
S315080011BC04D00026EFE7054E3400ECE72600EAE7F4
S315080011CC0026F0E7540200200028000850000020F2
S315080011DCF8B5CE46474680B505000C0016001F002C
S315080011EC4B0A5B029846036801330CD02B684345BF
S315080011FC10D1012399464B46012B14D04846C0BC46
S3150800120CB946B046F8BD4146FFF770FF814600283F
S3150800121CF1D0EBE741462800FFF7B2FF051E1FD0B9
S3150800122C01239946E7E72B68E41A2C19043406E0DF
S3150800123C3378237001340136013F002FDED000F0DD
S3150800124C52FB291D611A80239B009942F0D3190081
S3150800125C41442800FFF794FF051E04D0041DE7E758
S3150800126C00239946CAE700239946C7E710B5040038
S3150800127C80231B0598420DD3F8231B069C46644411
S3150800128C094B1B689B02FF22920213409C4206D212
S3150800129C042010BD0549064800F068FAECE7054934
S315080012AC034800F063FAF3E7E075FF1FAE0300008E
S315080012BC0C1E0008AF03000070B5040080231B0544
S315080012CC984211D3F8231B06E5180D4B1B689B0295
S315080012DCFF22920213409D420BD22000FFF7C6FF55
S315080012EC04280BD0002070BD0649074800F03EFACA
S315080012FCE8E70649044800F039FAEEE7E80AF2E7A7
S3150800130CE075FF1FCD0300000C1E0008CE0300007D
S3150800131CF0B587B00C0000230593884205D804283D
S3150800132C3DD912293DD8012700E00027012F02D00C
S3150800133C380007B0F0BDFFF7A1FE05002000FFF747
S3150800134C9DFE06002000FFF7B5FE3618013E761BFB
S3150800135C0136F60AB6B202230193013B0493FFF752
S3150800136C07FA0024B44217D22800FFF7A5FF03900A
S3150800137C2800FFF77BFF029000F0B5FA05A901A833
S3150800138CFFF79EFA002806D180231B019C4665446C
S3150800139C0134A4B2E6E70027FFF702FAC8E70027EC
S315080013ACC6E70027C4E7000001235B42024A136024
S315080013BC024A13607047C0465000002054020020B1
S315080013CC70B504000D0016004A1E124B1B1A9A42E1
S315080013DC01D9002070BDFFF72DFEFF2811D0281962
S315080013EC0138FFF727FEFF280BD0630A5B020A4A6F
S315080013FC934208D02B00320021000848FFF7E8FE7C
S3150800140CE8E70020E6E72B00320021000448FFF746
S3150800141CDFFEDFE7FFFF0108002800085000002068
S3150800142C5402002070B505000C004A1E0F4B1B1AFF
S3150800143C9A4205D9FF21FF260020012812D070BD3B
S3150800144CFFF7F8FD060060190138FFF7F3FD0100F8
S3150800145CFF2E03D0FF2803D00120EEE70020ECE78F
S3150800146C0020EAE73000FFF753FFE8E7FFFF010823
S3150800147C00B583B0104B1B68013302D1012003B0B1
S3150800148C00BD0D4A536891688C466344D1688C46F6
S3150800149C634411698C46634451698C46634491696B
S315080014AC8C466344D2699B185B42019301AA0421BA
S315080014BC0248FFF785FFE2E754020020BC28000823
S315080014CC0E4B1A680E4B1B68D2180E4B1B689A18D3
S315080014DC0D4B1B689B180D4A1268D3180C4A1268D8
S315080014ECD2180C4B1B689A180B4B1B689B18002BB5
S315080014FC01D1012070470020FCE7C04600280008EF
S3150800150C04280008082800080C28000810280008D9
S3150800151C1428000818280008BC28000810B50B4B1E
S3150800152C1B68013305D10A4B1B68013307D101200F
S3150800153C10BD0648FFF7EBFD0028F9D0F3E7044881
S3150800154CFFF7E5FD0028F3D00120F1E7540200204F
S3150800155C50000020004870470028000810B5FFF717
S3150800156C23FF10BD10B5FFF72BFF10BD10B5FFF705
S3150800157C59FF10BD10B5FFF7A3FF10BD10B5FFF747
S3150800158CE9FF10BD10B5FFF773FF002800D110BD99
S3150800159CFFF7C4FFFBE70000054BDB699B0604D588
S315080015AC034B5B6A0370012070470020FCE7C046BA
S315080015BC0044004010B5084B986200F0CBF80A308E
S315080015CC0400054BDB691B0605D400F08CF900F00A
S315080015DCC1F8A042F5D910BD0044004030B589B019
S315080015EC0C4C23680125AB432360E1231B020193B2
S315080015FC00230293039304930C22059206930793F4
S3150800160C009369462000FFF73FFC23682B432360B1
S3150800161C09B030BD0044004070B506000D004029E5
S3150800162C0ED82800FFF7C6FF0024ABB2A3420CD98C
S3150800163C00F059F9305DFFF7BDFF0134A4B2F4E7A9
S3150800164C7621024800F092F8EBE770BD001F0008FF
S3150800165C70B506000D00264B1C78002C17D12548B2
S3150800166CFFF79AFF012801D0200070BD214B1B788B
S3150800167C013BDBB23F2BF7D800F06CF81E4B186019
S3150800168C1E4B00221A701A4B01321A70ECE71B4BD0
S3150800169C1B7801331748C018FFF77EFF0400012892
S315080016AC17D1164B1A780132D2B21A70114B1B7815
S315080016BC9A4201D00024D7E792B20E490131300084
S315080016CCFFF7A8FC0A4B00221A700C4B1B782B70E0
S315080016DCCAE700F03FF8084B1B686433984204D9F4
S315080016EC034B00221A700024BEE70024BCE7C04650
S315080016FC99040020580400209C0400209A04002019
S3150800170C024B00221A605A609A60704710E000E09B
S3150800171C10B5FFF7F5FF054B054A5A6000229A608B
S3150800172C05211960034B1A6010BDC04610E000E095
S3150800173CFFF90000A0040020044B1B68DB0303D54B
S3150800174C034A1368013313607047C04610E000E083
S3150800175CA004002010B5FFF7EFFF014B186810BD69
S3150800176CA004002010B5FFF7F5FF10BD10B500F06A
S3150800177CBAF8FCE710B500F0ABF8012803D00B4B10
S3150800178C1B78012B00D010BDFFF7E4FF084B1B6834
S3150800179C084A12689B18F533FF339842F3D3034B68
S315080017AC00221A70FFF714FCEDE7C046A8040020C7
S315080017BCA4040020AC04002010B5054B1B78012BA3
S315080017CC00D010BDFFF7C6FF024B1860F9E7C046FC
S315080017DCA8040020AC04002010B5044B01221A7092
S315080017ECFFF7EAFFFFF7C6FF10BDC046A8040020A6
S315080017FC10B5FFF7E9FB00F072F8FFF789FFFFF762
S3150800180CADFE00F00DF8FFF7E7FF10BD10B500F0C0
S3150800181C6AF8FFF791FF00F00FF8FFF7ABFF10BD62
S3150800182C10B500F0D7F9FFF7D9FE024B00221A7053
S3150800183C10BDC0460C00002000B583B06B46D91D00
S3150800184C0748FFF705FF012801D003B000BD054B7B
S3150800185C00221A706B46D979014800F0D9F9F4E7D9
S3150800186CB00400200C0000207047000010B5054B92
S3150800187C1B78002B02D000F0C3F910BDC9B2FFF7D4
S3150800188CCBFEF8E70C000020074B1B78022B07D081
S3150800189C032B07D0012B01D0402070470020FCE712
S315080018AC0020FAE70020F8E70C000020074B1B780D
S315080018BC022B07D0032B07D0012B01D040207047F1
S315080018CC0020FCE70020FAE70020F8E70C000020CF
S315080018DC10B500F08DF9002800D0012010BD10B508
S315080018ECFEF7ACFC10BD10B5FEF7ADFC10BD000044
S315080018FC014B00225A707047F0040020034BFE225D
S3150800190CDA701871BA3A022199527047F00400201D
S3150800191C10B5054C00232370FFF7EAFFFF23E3708D
S3150800192CBB3B0122E25210BDF0040020064BFF22FD
S3150800193CDA7000221A71597859719A71DA711A7219
S3150800194C4432062199527047F004002010B5002045
S3150800195CFFF7D4FF10BD0000094BFF22DA70094AC5
S3150800196C9A6400221A715A719A710721D971002149
S3150800197C1972597299724422083199527047C046A5
S3150800198CF004002024200008044BFF22DA70426879
S3150800199C9A644422012199527047C046F0040020EB
S315080019AC10B53120FFF7AAFF10BD000070B5084C22
S315080019BCFF23E370002525716571FFF765FFA0719C
S315080019CCE5712572657244230722E25270BDC04642
S315080019DCF004002070B5FFF78BFF0D4C0125257020
S315080019ECFF23E370EF3B237100236371FFF74CFF72
S315080019FCA071FFF75BFFE071FFF758FF000A207232
S31508001A0C6572A57244230822E252FFF7A7FD70BD42
S31508001A1CF004002070B50400FFF736FF6278904298
S31508001A2C10D90A4D281DA96CFFF7F4FAFF23EB70A1
S31508001A3C6378AA6C94466344AB6463780133442296
S31508001A4CAB5270BD2220FFF759FFFAE7F0040020CD
S31508001A5C70B50400FFF718FF6378984212D96168CD
S31508001A6C0A4DA9646278281DFFF7D4FAFF23EB7098
S31508001A7C6378AA6C94466344AB6463780133442256
S31508001A8CAB5270BD2220FFF739FFFAE7F0040020AD
S31508001A9CF8B50500170000244E1E002907D02B7830
S31508001AAC1C19E4B20135FFF71EFF3100F4E73C6060
S31508001ABC0120F8BD10B5084CFF23E370E21D416800
S31508001ACCA06CFFF7E5FF207100236371A371443303
S31508001ADC0822E25210BDC046F004002070B504007E
S31508001AEC0E4B9D6CFFF7D0FE411E621C2800FFF7BB
S31508001AFC39FD00280DD0094CFF23E370FFF7C4FE0F
S31508001B0C0138A36C9C466044A06444230122E2522B
S31508001B1C70BD3130FFF7F2FEFAE7C046F00400203C
S31508001B2C10B50400FFF7B0FE01386378984216DD4D
S31508001B3C134BFF22DA70BB3A0121995261780029BE
S31508001B4C11D00F4B986CA21CFFF70CFD002812D075
S31508001B5C63780B4A916C8C466344936410BD2220BF
S31508001B6CFFF7CCFEFAE7FFF70DFD0028F6D131306A
S31508001B7CFFF7C4FEF2E73130FFF7C0FEEEE7C046CA
S31508001B8CF004002010B5094B9B6C41681800FFF750
S31508001B9CEDFC002806D0054BFF22DA70BB3A012172
S31508001BAC995210BD3130FFF7A9FEFAE7F004002070
S31508001BBC10B5FFF70DFA034BFF22DA70BB3A012179
S31508001BCC995210BDF004002010B589B2FFF74EFEED
S31508001BDC10BD0000054B00221A709A6443215A5412
S31508001BEC01315A529A705A707047C046F004002058
S31508001BFC024B1878002800D001207047F00400200A
S31508001C0C024A43230021D1547047C046F0040020F1
S31508001C1C10B50378FF2B0BD0294A1278012A13D159
S31508001C2C3733DAB2352A3AD89300264AD3589F4620
S31508001C3CFFF7D0FE224A4323D35C012B33D0204A2C
S31508001C4C4423D15E002932DC10BDFFF7E3FEF1E731
S31508001C5CFFF7FEFEEEE7FFF797FEEBE7FFF72AFF27
S31508001C6CE8E7FFF779FEE5E7FFF770FEE2E7FFF72F
S31508001C7C5DFEDFE7FFF74CFEDCE7FFF72FFFD9E742
S31508001C8CFFF74EFFD6E7FFF791FED3E7FFF77AFF8C
S31508001C9CD0E7FFF78DFFCDE7FFF782FECAE72020D6
S31508001CACFFF72CFEC6E71020FFF728FEC7E7100043
S31508001CBC43230122C2540330FFF786FFC4E7C0460C
S31508001CCCF00400204C1F000870B500260C4D0D4C76
S31508001CDC641BA410A64209D1002600F021F80A4D6F
S31508001CEC0A4C641BA410A64205D170BDB300EB5870
S31508001CFC98470136EEE7B300EB5898470136F2E7FA
S31508001D0C2C2000082C2000082C2000083020000865
S31508001D1C03008218934200D1704719700133F9E712
S31508001D2CF8B5C046F8BC08BC9E467047F8B5C04620
S30D08001D3CF8BC08BC9E4670477E
S31508001D4410B50C4A54698023DB0223435361EFF32D
S31508001D54108472B6002303E004C904C00133DBB25D
S31508001D643F2BF9D9034B1B69DB03FBD484F3108897
S30D08001D7410BDC0460020024024
S31508001D7C0000000000000000000000000000000049
S31508001D8C0000000000000000000000000000000039
S31508001D9C010000000200000003000000040000001F
S31508001DAC06000000070000000800000009000000FB
S31508001DBC0000000000000000000000000000000009
S31508001DCC01000000020000000300000004000000EF
S31508001DDC01000000020000000400000006000000DC
S31508001DEC080000000A0000000C00000010000000AB
S31508001DFC20000000400000008000000000010000E8
S31508001E0C433A2F576F726B2F736F667477617265CF
S31508001E1C2F4F70656E424C545F53544D33324730D6
S31508001E2C5F43414E2F5461726765742F536F7572F9
S31508001E3C63652F41524D434D305F53544D333247F2
S31508001E4C302F666C6173682E63000000002800084A
S31508001E5C000800000500000000300008000800001B
S31508001E6C0600000000380008000800000700000003
S31508001E7C00400008000800000800000000480008A0
S31508001E8C00080000090000000050000800080000C7
S31508001E9C0A00000000580008000800000B000000AB
S31508001EAC00600008000800000C000000006800082C
S31508001EBC000800000D000000007000080008000073
S31508001ECC0E00000000780008000800000F00000053
S31508001EDC00800008008000001000000000000108C7
S31508001EEC008000001100000000800108008000003E
S31508001EFC12000000433A2F576F726B2F736F66747C
S31508001F0C776172652F4F70656E424C545F53544D12
S31508001F1C333247305F43414E2F5461726765742FD5
S31508001F2C536F757263652F41524D434D305F535451
S31508001F3C4D333247302F72733233322E6300000022
S31508001F4C861C0008AA1C0008AA1C0008A41C000869
S31508001F5CAA1C0008AA1C00089E1C00088C1C000859
S31508001F6C981C0008921C0008AA1C0008AA1C000849
S31508001F7CAA1C0008AA1C0008AA1C0008AA1C00080F
S31508001F8CAA1C0008AA1C0008AA1C0008AA1C0008FF
S31508001F9CAA1C0008AA1C0008AA1C0008AA1C0008EF
S31508001FACAA1C0008AA1C0008AA1C0008AA1C0008DF
S31508001FBCAA1C0008AA1C0008AA1C0008AA1C0008CF
S31508001FCCAA1C0008AA1C0008AA1C0008AA1C0008BF
S31508001FDCAA1C0008AA1C0008AA1C0008AA1C0008AF
S31508001FECAA1C0008AA1C0008681C00085C1C00082F
S31508001FFC561C0008621C0008AA1C0008AA1C00082B
S3150800200CAA1C00086E1C0008AA1C0008741C0008F0
S3150800201C7A1C0008801C00084F70656E424C5400F0
S3090800202CE5000008B5
S30908002030BD000008D9
S315080020340024F4000100000004000000040000006D
S7050800059D50
